:1000000012C017C016C015C014C013C012C011C052
:1000100010C00FC00EC00DC00CC00BC00AC009C07C
:1000200008C007C006C011241FBECFEDCDBF28D029
:1000300046C0E6CF12B88DE489B9599886E083B9F5
:1000400088E18AB908955D9BFECF8CB908955F9BC6
:10005000FECF8CB10895CF93C82F982F92959F70A3
:100060009A3010F480E301C087E3890FECDF8C2F16
:100070008F708A3010F4805D01C0895CCF91E3CF2E
:100080002FE088E190E00FB6F894A89581BD0FBEEF
:1000900021BD10BE84E083BFBA9AC298CBDFC0E016
:1000A00012E0D4E0A89508B601FEFCCF18BFCF5FE0
:1000B000C9F788B38D2788BB88E4C5DFF3CFF894F0
:0200C000FFCF70
:00000001FF
